:020000000528D1
:10000A0010308316850083128316860183128F01AE
:10001A000A30900091010A309200C320F6200000B5
:10002A00051E1828152801308F000F08013C031DF2
:10003A001F28EA200F08013C03192628031826283E
:10004A00E420FC20051E2A2832288F0A0F08103CBB
:10005A00031D312801308F001A280230910011083F
:10006A00013C031D3928F6201108013C03194028D8
:10007A0003184028F0201321051A44284C28910A15
:10008A0011080A3C031D4B28013091003428051A37
:10009A004F284C280F080F3C031D88281108073CDD
:1000AA00031D8828C320F620EA200A309000FC208D
:1000BA0001308F006A28E420FC20051A67280F08FF
:1000CA0090006F280F08013E8F000E3C031960282C
:1000DA00031860281008033C03197728031C7728A3
:1000EA0002309000023010029000100810079000B1
:1000FA0010081007900010080F07023C003C9000FF
:10010A000A30100790000F080F3C031DBF28110882
:10011A00083C031DBF28C320F620EA20FC2001303A
:10012A008F00A128E420FC20051A9E280F089200BF
:10013A00A6280F08013E8F000E3C031997280318C2
:10014A0097281208033C0319AE28031CAE28023074
:10015A00920002301202920012081207920012084C
:10016A001207920012080F07023C003C92000A3064
:10017A0012079200051AC228BF281228051001305A
:10018A008C00CC28051105150C08013E8C00093C91
:10019A000319C7280318C7288514851005100130CC
:1001AA008C00DC28061006140C08013E8C000F3C5B
:1001BA000319D7280318D7288614861008000510B3
:1001CA000610061486148610080005140610061474
:1001DA00861486100800051005110515851485106A
:1001EA000800051405110515851485100800100866
:1001FA008D008D0301308C00062900000C08013E99
:10020A008C00503C03190229031802290D08003CEE
:10021A000319122903181229FE28080012088D0052
:10022A008D0301308C001D2900000C08013E8C0052
:10023A00503C03191929031819290D08003C031900
:0A024A0029290318292915290800A5
:00000001FF
